:10000000A0019D2990002408840022081021841357
:100010000005181C2206031920281008031D1828A3
:100020001608FF3E031C21280A3025211608212826
:10003000100AFF3003192028100B20281708212848
:100040009909990C9829A016A01EA01220192D28F4
:10005000FE39A100201503109829201A3528920096
:1000600020164C2003183A281208532003183A2867
:10007000A01E982945206A2020112012A0112408D2
:1000800084002208841780044B2824088400220955
:1000900080058417800508003F206A2045206620DF
:1000A0002108A01901388E0008308F008E0D03182A
:1000B0003F20031C45206A2066208F0B56283F20D6
:1000C0006A202408840022080005FF3E25088400D9
:1000D000230948282508840023088004841723095D
:1000E00080054B2891019000A11727308F00103018
:1000F000852003308F00E83085208F016430852013
:100100008F010A308520100890288E0011088D007C
:1001100010088C0061210C08031DA113A11B08000D
:10012000303E9328040893008611861086108316AB
:100130008611861086100F30860583121308A018CA
:10014000BF283A308D009830332133309200D320CD
:1001500013308D0088303321D32064303221D320F6
:100160006430322122309200D3202030BE200C3067
:10017000BE200630BE20A0141308BF282014920011
:10018000201CCD288610033C031CD228D220073027
:100190008D00D0303321031408002014FE3C0319D5
:1001A00098298614201C201086150F308605120809
:1001B000F03986048611920E2018D328323032216D
:1001C00003140800A11315080319A11705309400A2
:1001D00027308F001030F82003308F00E830F820EF
:1001E0008F016430F8208F010A30F8201008FF28B2
:1001F0008E0011088D0010088C0061210C088C0005
:1002000094030319A11315080319092914020318EB
:1002100008000C08031DA113A11B0800303E932900
:10022000841780049829890083160814831208080B
:10023000982988008316081555308900AA3089004E
:10024000881488182129081198298F018E00FF3001
:100250008E07031C8F07031C982903308D00DF30A5
:10026000332127298D01E83E8C008D09FC30031CC9
:100270003C298C07031839298C0764008D0F392914
:100280000C1842298C1C46290000462908008E00C3
:10029000023051298E00063051298F018E00043022
:1002A000512994000F080D02031D58290E080C0255
:1002B000043003180130031902301405031DFF3008
:1002C000982991019001103092000D0D900D910D23
:1002D0000E0890020F08031C0F0F910203187729D4
:1002E0000E0890070F0803180F0F910703108C0DCD
:1002F0008D0D920B65290C089829103094008D0102
:100300008C01930C920C031C8B290E088C070F0890
:1003100003180F0F8D078D0C8C0C910C900C940B07
:1003200081291008982984001D088A001C08820071
:1003300083130313831264000800831605148514C5
:100340000515051685158312C230B4008030AE0045
:100350003E30AF000130BB0064302521061183160A
:100360000611FE30831293200130932054309320E5
:1003700058309320203093204130932054309320E4
:100380005630932020309320323093202E3093200B
:100390003330932047309320483093207A30932095
:1003A000203093207630932030309320BC014130B0
:1003B000B200B30103308F00E83026213C0813213E
:1003C000B00001303C079E009F019F0D1E081321C5
:1003D000B1002E083007AC002F080318013E31078A
:1003E000AD000630A4000130A2000630A5000230A6
:1003F000A300340825202D0825202C0825208E3028
:100400002320C322EE2201308F00F4302621053054
:10041000A4000830A2009801FF3096009701013037
:10042000990039080220B9000318672A0530A40092
:100430000830A20001309800FF309600970101308B
:1004400099003A080220BA0003186C2A0530A4006B
:100450000130A20098010A30960002309700013066
:10046000990035080220B5000318722A0530A4004F
:100470000230A20098010A30960002309700013045
:10048000990036080220B6000318832A0530A4001C
:100490000430A2009801FF309600970101309900C6
:1004A00038080220B8000318442B0530A40010308F
:1004B000A2009801FF30960097010130990037089B
:1004C0000220B7000318A12A64302521072ABC01A5
:1004D0004130B200B301DE290230BC004230B2002C
:1004E000B301DE293B08B0070318B10A30088C00BD
:1004F00031088D0014308F0050304A21031D822AAC
:10050000B001B101E92930088C0031088D003B08A9
:100510004D21031D9E2A30088C0031088D008F016B
:1005200000304721031D992A3B08B002031CB10388
:10053000E9295030B0001430B100E929B001B1010F
:10054000E92964003B08503C0319B72A64003B08C2
:10055000083C0319BD2A3B089200930102308E002B
:100560008F017D21BB001723C322EE22072A013011
:10057000BB001723C322EE22072A5030BB001723EB
:10058000C322EE22072A80302C02A6003E30031C34
:10059000013E2D02A70026088C0027088D00083098
:1005A0008E008F016121A8000D08A90026088C008B
:1005B00027088D0008308E008F01612110089E00F1
:1005C00011089F007D30920093011E088E001F08C5
:1005D0008F007D21AA001108AB000800FE30932097
:1005E00001309320023072200330950028089000DB
:1005F0002908910092309C009D01E2202E3093202A
:10060000033095002A0890002B08910092309C003E
:100610009D01E220203093204D30932048309320DC
:100620007A30932020309320320893200800FE3047
:100630009320013093205030932061309320733009
:100640009320203093206430932065309320203015
:1006500093207D30920093013B088E008F017D2115
:100660009E0011089F001F0891001E087320203073
:1006700093206B309320483093207A3093200530BC
:100680008F00DC30262108003C0889003008192141
:1006900001303C079E009F019F0D1E088900310814
:1006A0001921FE30932001309320203093204D30CB
:1006B0009320453093204D3093204F30932052307B
:1006C000932049309320533093204530932020309D
:1006D0009320733093207530932072309320203014
:1006E00093203208932005308F00DC302621C3226E
:0406F000EE22072AC5
:02400E00F53F7C
:08420000A000090000000A0003
:00000001FF
